:0200000480007A
:100000006F000005732F2034930F80006308FF03F7
:10001000930F90006304FF03930FB0006300FF038E
:10002000130F000063040F0067000F00732F2034CC
:1000300063540F006F00400093E19153171F0000BD
:1000400023223FFC171F000023200FFC6FF01FFF2F
:100050009300000013010000930100001302000050
:100060009302000013030000930300001304000038
:100070009304000013050000930500001306000020
:100080009306000013070000930700001308000008
:10009000930800001309000093090000130A0000F0
:1000A000930A0000130B0000930B0000130C0000D8
:1000B000930C0000130D0000930D0000130E0000C0
:1000C000930E0000130F0000930F0000732540F102
:1000D0006310050097020000938202017390523072
:1000E000735044749702000093820201739052305F
:1000F00073500018970200009382420273905230AE
:100100009B021000939252039382F2FF7390023B82
:100110009302F0017390023A73504030970200004E
:1001200093824201739052307350203073503030BC
:100130009301000097020000938202ED7390523009
:10014000130510001315F501635C05000F00F00F97
:10015000930110009308D005130500007300000000
:1001600093020000638A020073905210B7B200003D
:100170009B829210739022307350003097020000DF
:100180009382420173901234732540F17300203042
:1001900093012000B70000801BD70000B703008048
:1001A0006310773293013000B70000801BD7100036
:1001B000B70300406316773093014000B70000801A
:1001C0001BD77000B7030001631C772E930150000A
:1001D000B70000801BD7E000B70302006312772E40
:1001E00093016000B70000809B8010001BD7F001D6
:1001F000930310006316772C930170009300F0FFB7
:100200001BD700009303F0FF631C772A9301800043
:100210009300F0FF1BD71000B70300809B83F3FF10
:100220006310772A930190009300F0FF1BD77000B2
:10023000B70300029B83F3FF631477289301A000A8
:100240009300F0FF1BD7E000B70304009B83F3FF8C
:10025000631877269301B0009300F0FF1BD7F001DD
:1002600093031000631E77249301C000B72021215F
:100270009B8010121BD70000B72321219B831312F0
:10028000631077249301D000B72021219B801012A6
:100290001BD71000B79390109B830309631277223A
:1002A0009301E000B72021219B8010121BD7700022
:1002B000B74342009B832324631477209301F0000B
:1002C000B72021219B8010121BD7E000B7830000CC
:1002D0009B8343486316771E93010001B7202121B9
:1002E0009B8010121BD7F00193030000631A771C48
:1002F0009301C002B720F1FF9B8050349390C0005F
:10030000938080671BD70000B75334129B838367A9
:100310006318771A9301D002B720F1FF9B80503405
:100320009390C000938080671BD74000B7432301A0
:100330009B837356631677189301E002B720090078
:100340009B8050349390C000938080671BD700003F
:10035000B75334929B838367631477169301F0023B
:10036000B72009009B8050349390C0009380806731
:100370001BD74000B74323099B837356631277143E
:1003800093011001B70000809BD07000B7030001FB
:10039000639870129301200113020000B7000080DF
:1003A0001BD77000130307001302120093022000F2
:1003B000E31652FEB703000163147310930130017A
:1003C00013020000B70000801BD7E00013000000FC
:1003D000130307001302120093022000E31452FEDD
:1003E000B7030200631E730C930140011302000067
:1003F000B70000809B8010001BD7F00113000000A5
:1004000013000000130307001302120093022000E0
:10041000E31052FE930310006314730A930150011A
:1004200013020000B70000801BD7700013021200F7
:1004300093022000E31852FEB7030001631277080D
:100440009301600113020000B70000801300000058
:100450001BD7E0001302120093022000E31652FEA5
:10046000B7030200631E77049301700113020000BA
:10047000B70000809B8010001300000013000000F4
:100480001BD7F0011302120093022000E31252FE68
:100490009303100063167702930180019B50F001D3
:1004A00093030000639E7000930190019300F0019C
:1004B0001BD0C0019303000063147000631030026E
:1004C0000F00F00F638001009391110093E1110080
:1004D0009308D00513850100730000000F00F00F92
:1004E000930110009308D00513050000730000006D
:0C04F000731000C00000000000000000BD
:1010000000000000000000000000000000000000E0
:1010100000000000000000000000000000000000D0
:1010200000000000000000000000000000000000C0
:1010300000000000000000000000000000000000B0
:081040000000000000000000A8
:040000058000000077
:00000001FF
